:020000000C945E
:100002006D010C94950B0C9400000C9400000C9460
:1000120000000C9400000C9400000C9400000C945E
:1000220000000C9400000C9429020C9400000C9423
:1000320000000C9400000C9400000C9400000C943E
:1000420000020C9400000C94F2080C9400000C9432
:100052003E090C9400000C9400000C9400000C94D7
:1000620000000C9400000C9400000C9400000C940E
:1000720000000C9400000C94680A0C9400000C948C
:100082004C0B0C9400000C940000000102040810B8
:100092002040800068010000801002006C01150001
:1000A200011000007A011300010100008201010029
:1000B200010200008C01020001020000960103000F
:1000C20001020000A001040001020000AA010500D3
:1000D20001020000B401060001020000BE01070097
:1000E20001020000C801080001020000D20109005B
:1000F20001020000DC010A0001020000E6010B001F
:1001020001020000F0010C0001020000FA010D00E2
:100112000102000004020E00010200000E020F00A4
:100122000102000018021000010200002202110068
:10013200010200002C021200010200000000000077
:10014200FF0000000000010002000400080010008F
:10015200200040008000000100020004000800109E
:100162000020004000805F4944005F53656E64498F
:100172006E707574546F00005F52656C6169730034
:100182005F496E7075745F3100005F496E707574FF
:100192005F3200005F496E7075745F3300005F4923
:1001A2006E7075745F3400005F496E7075745F35F0
:1001B20000005F496E7075745F3600005F496E70B3
:1001C20075745F3700005F496E7075745F380000A8
:1001D2005F496E7075745F3900005F496E707574A7
:1001E2005F3130005F496E7075745F3131005F4975
:1001F2006E7075745F3132005F496E7075745F3175
:1002020033005F496E7075745F3134005F496E7000
:1002120075745F3135005F496E7075745F313600F9
:100222005F496E7075745F3137005F496E70757427
:100232005F3138001027E80364000A000100001053
:1002420000011000010049530049430025642E2596
:10025200326400445300564300494C00235022416B
:10026200534349492D492F4F222C22312E3030221F
:100272002C323030382D30312D30313B00234822A2
:1002820045636F222C22312E3030222C323030380E
:100292002D30312D30313B0023532245636F222C08
:1002A20022312E3030222C323030382D30312D3068
:1002B200313B00002564002530325800253130647E
:1002C200000056430049500001002D4E414E0000EF
:1002D2000100E00FCA020000F894EE27ECBBF1E047
:1002E200F5BFE5BFE0936C00F8E1F1BDE1BD8DE043
:1002F200A2E0BB27ED938A95E9F780E090E1A0E0C8
:10030200B1E0ED930197E9F7E2EDF2E08591959185
:10031200009761F0A591B59105901590BF01F0018C
:1003220005900D920197E1F7FB01F0CFEFEFEDBFE2
:10033200E0E1EEBFC0E0D5E00C946503E09163001C
:10034200E0710895E881E03021F0E0916500EE7FF0
:1003520003C0E0916500E160E09365000C94E6045F
:10036200E6B3F0E0DF01E0B1FE2FE0E0EA0FFB1FB1
:100372000895E6B3E093920BA3E9BBE0E0B1EC93FE
:10038200E0B3E073E295EF70E093940B0895A091CF
:10039200DF0CB091E00CEFEFF0E0EA27FB27EBBBBC
:1003A200E091DF0CF091E00C0E94A615AFEFB0E0F7
:1003B200EA27FB27E5BB0E943704E87021F4E091AD
:1003C2006500E16003C0E0916500EE7FE0936500A7
:1003D200A3E1B0E00E941A16E13031F4E091DF0CA3
:1003E200F091E00CE17009F404C0E0916500E26074
:1003F20003C0E0916500ED7FE093650008950E94DF
:100402003713E4E6E2BF0E94100478944394E2E3D7
:10041200E41519F4E1E0E71509F002C07724442459
:10042200E2E3E41519F4E0E0E71509F003C0E1E0C6
:100432007E2E4424A0910105A13028F0E09101050F
:10044200E150E093010595DF0E94B30EA0DF0BC0DF
:100452000E943713E6E0E4BD83DFFA93EA930E9439
:10046200260E0E94D90DE991EFBFF991E991B99158
:10047200A9919991899179916991F990199009902D
:1004820018951A93A0915808A13051F4DA92CA92A1
:10049200E4E6F0E0FA93EA930E944304E03009F4C0
:1004A20009C0E0E0E0935808E3E0E91518F40E947F
:1004B20045139924A0915808A23041F4DA92CA92C5
:1004C2000E944D130E944304E03009F403C0E0E0AF
:1004D200E0935808A0915808A03059F4E0915106D1
:1004E200A0915206EA1729F0A0E020FCA1E0A0307A
:1004F20009F027C00E945213EE5FFA4FE081E1300B
:1005020039F40E9452130E9458130E945F1319C0BB
:10051200E23011F0E330A9F40E945213EE5FFA4F79
:10052200E081E23009F499240E9452130E94581388
:10053200EE5FFA4FA3E0A08399D16F01E1E0E0936F
:1005420058080C940F051A93A0915506A43011F483
:1005520010918A07A0915506A53011F41091F10768
:10056200143049F4E981E03011F4E0E001C0EFE039
:10057200EA930E948F04153049F4E981E03011F4C6
:10058200E5E101C0E6E0EA930E948F0462C01A939B
:10059200E3E0EA930E948F0410915406E12FE29562
:1005A200EF700E946413E12FEF700E946413E7E181
:1005B200EA930E948F040C940F05E2E0EA930E94F2
:1005C2008F04E0E0E0935406E9E4EA930E948F048A
:1005D200E881E05DEA930E948F04D9DFA09155067D
:1005E200A43011F40E946A130E9471131696E1E07E
:1005F200EC93E8810E9476130C94E6041A93A0917E
:100602005506A43011F40E946A1310E0173060F40A
:100612000E9471131A96EE27A10FBE1FEC91EA9366
:100622000E948F041F5FF2CFE981E03011F4E0E312
:1006320005C0E091060DF091070DE189EA930E9451
:100642008F040E9471131696E1E0EC93E9810E94F7
:100652007613188122960895E0915906A0915806C2
:10066200EA1759F0A0915706A13039F40E942D09DA
:10067200EB3018F063DEE03009F40FC0E091590668
:10068200F0E0E65AF94FE081EA930E946E09A091E8
:1006920059060E947D13E093590608951A93A8956E
:1006A2000E944A0D0E94140DECDED6DFE0E0E71551
:1006B20021F4A0910105A03011F0E1E001C0E0E0D9
:1006C200EA9340DE0C940F05E0E0E5BFE0936D0095
:1006D200E0936C00EFEFEBBBEABBE5BBE4BBE0E011
:1006E200E2BBE1BBE0936200E0936100E3B9E2B9EF
:1006F200E1E0E0936500E3E0E0936400E0E0E8BB62
:10070200E7BBE0BFE7E0E3BFE4E6E2BFE0E0E1BF72
:10071200EFBDEEBDEDBDECBDE7BDE6BDEBBDEABD97
:10072200E9BDE8BDE0937900E0937800E3E0E5BD40
:10073200E6E0E4BDE0E0E3BDE0938B00EAE0E093B5
:100742008A00E0E0E0938900E0938800E093810072
:10075200E0938000E2E1E0938700E4E3E093860027
:10076200E0E0E0938500E0938400E0938300E0936F
:100772008200E0936A00EABFE9BFE1E4E7BFE0E09C
:10078200E0937D00EBB9E8EDEAB9E6E0E09395008D
:10079200E0E0E0939000E6E6E9B9E0E0E0939B0058
:1007A200E8EDE0939A00E6E0E0939D00E0E0E0935C
:1007B2009800E3E3E0939900E0E8E8B9E0E0E0BD07
:1007C200EEE1E1BDEEE0E1BD0E94CD080E94201104
:1007D2000E948213E53128F0A0E0B0E0E0E00E9440
:1007E2002E16A8950E94871388240E9482138E16C3
:1007F20048F4A895E1E00E948D13E0E00E948D1379
:100802008394F3CF0E9487137894EFEF6E2E46DF26
:100812000E94E410E1E0E0935706F9CFFFCFA8E091
:10082200BDE00E9496130895A881A03310F0AA3368
:1008320008F003C0E881E053C8C0A881A13410F0D9
:10084200A73408F003C0E881E753BFC0EFEFBDC093
:10085200A881AA3018F4E881E05DB7C0A881AA3067
:1008620018F0E881E95CB1C0E8E5AFC01A930A93D9
:10087200F8940091080D1091090D7894F8010991EE
:10088200199108951A930A93F1DF8F01EA81FB818E
:10089200AC81BD81EA0FFB1FE01BF10BDF010E945F
:1008A2003F1624F4E0E019810881E9C2E1E01981F0
:1008B2000881E5C2E881EF5FE883A881A53010F0E6
:1008C200E0E0E883E88181C0A0915206BB27E09175
:1008D2005106F0E031960E949C133596DF01E5E067
:1008E200F0E00C943B09A0915906BB27E091580611
:1008F2000C943209A0915306A13059F4A0915706E5
:10090200A13039F4F0DFE93220F00E949F01E0309B
:1009120009F402C0E1E00895E0E00895E881A091C1
:100922005406EA27E0935406E0915506E13071F44B
:10093200E0915806F0E0E65AF94FA881A083A09111
:1009420058060E947D13E09358063FC0E23071F4CE
:10095200E091BE06F0E0E054F94FA881A083A09197
:10096200BE060E947D13E093BE062FC0E33071F4F1
:10097200E0912407F0E0EA5DF84FA881A083A091FE
:1009820024070E947D13E09324071FC0E43071F412
:10099200E0918B07F0E0E357F84FA881A083A09184
:1009A2008B070E947D13E0938B070FC0E53069F43B
:1009B200E091F207F0E0EC50F84FA881A083A091FB
:1009C200F2070E947D13E093F20721960895E091C9
:1009D2005C0BEA930E94300CE0915D0BEA930E945B
:1009E200300C0895F4DF0E94A1130E94A113E88144
:1009F200F9810E94AB130C9495091A930E94040C7E
:100A02001E2F103021F0E12FE150E0935B0BDFDF6E
:100A1200E0915B0BEF5FF0E00E94AB131991089538
:100A220028970E94431650E00E94C70BE13010F451
:100A32000C946306E0915C0BE43411F00C94920583
:100A4200E0915D0BE33221F40E94040CE093530623
:100A5200E0915D0BE33549F4E5E5F2E00E94B31362
:100A620049DFE05DEA930E94300CE0915D0BE035D6
:100A720011F00C949105E2E2EA930E94BB0BE03084
:100A820019F0AF85A13009F04BC020E00E94B713E6
:100A9200A03240F00E94B713A23221F00E94B71395
:100AA200AB3309F43DC0E22FE03071F40E94B7137A
:100AB200A33211F421E007C0E0915306E0935506FA
:100AC2000E94BD132BDF29C0E13049F40E94B71305
:100AD200A43211F422E001C020E010E01EC0E23096
:100AE20011F0E330D1F40E94BD139EDEEF3FA1F07E
:100AF200E12FE295E07F4E2F0E94BD1395DEE40FB9
:100B02001E2F2F5F243039F4E0915306E0935506EF
:100B12001A9304DF20E001C020E00E94C413B6CF84
:100B2200CEC0E63511F00C944706E0915D0BE3343C
:100B3200B1F50E94C71330E0303188F50E94CD1321
:100B4200E156F44FE0811E1741F5AFEDBBE0EE2711
:100B5200A30FBE1FAC91A230D9F4E8E5F2E00E94E7
:100B6200B313E12F0E94D0130E94D613AFE4BCE06E
:100B72000E94CD130E94DA130E94E1130E94D61341
:100B8200AFE6BCE00E94CD130E94DA130E94AB13C1
:100B92000E94CD130E94E51302C03F5FCDCFE091CA
:100BA2005D0BE33511F00C9417060E94040CE093E0
:100BB200970B0E94EA13C9F50E94040CE093980B6C
:100BC2000E94EA1391F50E94040CE093990BE03025
:100BD20019F0E1E0E093990B0E94EA1331F50E94CB
:100BE200040CE0939B0BF0939C0B0E94EA13E9F434
:100BF2000E94040CE0939D0BF0939E0B0E94EA135B
:100C0200A1F40E94C713EE85E0939A0BE0E0EA9309
:100C12001A930E94EC0FE03041F4E8E5F2E00E9402
:100C2200B3130E94F0130E94AB1349C0E0915D0B15
:100C3200E53559F50E94C7130E94EA1329F50E946F
:100C4200040C0E2F30E03031F8F40E94CD13E1563F
:100C5200F44FE0811E17B1F4013049F4AFECBBE070
:100C62000E94CD130E94F313E068D001EC93003090
:100C720049F4AFECBBE00E94CD130E94F313EF776F
:100C8200D001EC933F5FDFCF1AC019C0E934B9F449
:100C9200E0915D0BEC3499F4EBE5F2E00E94B313C2
:100CA200E091920B0E94FD13E091930B0E94FD13C1
:100CB200E091940BF0E0FA93EA930E946E0C0E948A
:100CC200A80BB2CE0E940314609608950E944316A8
:100CD2000E94C70BE13010F40C943E07E0915C0BCC
:100CE200E33211F5E0915D0BEC3431F4E4E0E09392
:100CF200E10CE0E0E093760BE0915D0BE43599F4D2
:100D0200E091760BE03029F0EF77A0E0B0E00E94AE
:100D12002E160E944D130E948B15E0E0E093760B95
:100D2200E7E0E093E10C04C0E43511F00C943B07DA
:100D3200E0915D0BE33231F40E94040C3197E093B1
:100D42005B0B98C0E03511F00C943B0710E00E9459
:100D5200B713A03250F00E94B713AD3331F00E94A6
:100D6200B713AB3311F01E3008F00CC00E94F01321
:100D7200E25AF44F0E940C14D001EC931F5F0E94C0
:100D8200C413E5CF0E94F013E25AF44FA0E0A0830F
:100D9200EDE3EA930E94BB0BE13011F00C943B07A8
:100DA200E4E5E093720B10E00E94F0130E9413142A
:100DB2003496E491EF3F11F40C943B070E9418140F
:100DC2000E94F0130E9413140E940616FA93EA93EB
:100DD2000E948611E03011F00C9439070E94F01342
:100DE2000E9413143496E491E03839F40E94040C02
:100DF200E058FF4FE093760B3BC0E03011F0E1305A
:100E0200A1F40E94F0130E94131432960E94061657
:100E1200FF93EF930E94040CAF91BF910E942E1694
:100E22000E944D130E948B1523C0E23081F40E9470
:100E3200F0130E94131432960E940616FF93EF934A
:100E42000E94040CAF91BF910E94261611C0E3309C
:100E520079F40E94F0130E94131432960E9406162F
:100E6200FF93EF930E94E30BAF91BF910E942E1666
:100E72001F5F9ACF0E94A80B2BCF0E9403142696C5
:100E820008950E9445160E94C70BE13010F40C949D
:100E9200B707E0915C0BE332A9F4E0915D0BE0351A
:100EA20019F4EEE5F2E009C0E83419F4EFE7F2E0F4
:100EB20004C0E33531F4EAE9F2E0FA93EA930E94DE
:100EC200410C51C0E43511F00C94B407E0915D0B74
:100ED200E43231F4E5E1F0E0FA93EA9383DD43C0D2
:100EE200E33211F48ADD3FC0E035E9F570DDA0910F
:100EF2005B0BA531C0F50E941D140E9406160E94CC
:100F0200B313EDE3EA930E94300C0E941D14349651
:100F1200E491E03829F40E9482130E94211423C034
:100F2200E03011F0E13049F40E941D140E942314B4
:100F32000E941A160E94211416C0E23049F40E943F
:100F42001D140E9423140E9416160E94E1130BC066
:100F5200E33049F40E941D140E9423140E941A16C1
:100F6200EA930E947C0C0E94A80B8DCF0E94281449
:100F7200E0E0EC930E944C16249608951A930A938B
:100F820000E0A0915808A13081F40E945213EE5F54
:100F9200FA4FE081E33049F40E945213EB5FFA4FBB
:100FA200E381A0915E0AEA1709F03FC00E942D1466
:100FB20001E00E94C70BE130A0F1E0915C0BE2344A
:100FC20079F5E0915D0BE13459F50E94040C1E2F76
:100FD2000E945213ED5FFA4FE081E09355060E94A2
:100FE2005213EC5FFA4FE081E73419F41A930E942E
:100FF200A4020E945213EC5FFA4FE081E33419F429
:101002001A930E94DE020E945213EC5FFA4FE081B3
:10101200E53419F41A930E94FF02EEE1E093010510
:10102200C8CF0E9452130E945F13E02F0C94010C50
:101032001A930A930E942D1447DCE23078F10E9441
:1010420034140E943A140E9447140E942814E2E7C2
:101052000E944E14E0915E0A0E9452140E9454149F
:10106200A0915E0AE0910A0DEA1721F4E0915E0A6E
:10107200E03311F401E001C000E0E0915E0AE09388
:101082000A0D0A93E0915C0AEA93CADC0E945714A3
:101092000E9434140E945B140C94010CE0E00C9446
:1010A200010C1A93EBE5F9E00E946814EBE5F8E015
:1010B2000E946D140E9457140E947214E181E4345C
:1010C20071F40E94721402800E948213E05DE015A6
:1010D20029F00E947214E281EA3209F401C028C0A8
:1010E2000E9477140E947214E1810E9452140E949D
:1010F2007214E2810E9452140E947A141C910E947E
:10110200721433960E946D14E12FE23139F40E9479
:1011120028141397E6E0EC93D9DD08C0E13131F4ED
:101122000E9428141397E2E1EC93ABDE0E94980C24
:101132000C94600C1A93C8DBE23058F10E9434140C
:101142000E943A140E9447140E942814EAE70E945F
:101152004E14EFE5FAE00E946D140E947A14119782
:101162001C91E12FE23131F4E6E0EA930E94300C67
:10117200ADDD07C0E13129F4E2E1EA930E94300CCF
:1011820080DE0E9457140E9434140E945B140C9457
:10119200600CE0E00C94600CEFEFE093720BE093D4
:1011A200730B0895AC81A03310F0AA3308F006C087
:1011B2000E947F14E0530E9487140FC0AC81A134B7
:1011C20010F0A73408F006C00E947F14E7530E9473
:1011D200871403C0A881B981E0E0EC9325960895B5
:1011E200EDC2AA93EA93FA93EFB7EA931A930A939A
:1011F2001BB10CB1E0914A0DF0E0E85EF24F0083C2
:10120200A0914A0DAF5FA0934A0DA23319F4E0E01A
:10121200E0934A0D099119915CC21A93E0914B0D2A
:10122200A0914A0DEA17D1F3F0E0E85EF24F108187
:10123200A0914B0DAF5FA0934B0DA23319F4E0E0E8
:10124200E0934B0DE12F3BC3E0914B0DA0914A0D72
:10125200EA1709F0B3C2B4C2A091B10DBB27E09165
:10126200B00DF0E031960E949C13EC59FF4FDF0164
:10127200E4E6F0E00E94E61508950E943713E0913B
:10128200B10DA091B00DEA1741F0A0915706A03020
:1012920019F0A6DFE03009F001C011C0E091B10DF4
:1012A200F0E0E45BF24FE081ECB9A091B10DAF5FE9
:1012B200A093B10DA43619F4E0E0E093B10DE991E9
:1012C200EFBFF991E991B991A99199918991799198
:1012D2006991F9901990099018951A93E091B10DBE
:1012E200A091B00DEA1751F45D9B08C0A09157067A
:1012F200A13019F475DFE03009F013C01091B00D80
:101302000E94F013E45BF24FA981A0831F5F1436A1
:1013120009F410E0E091B10DE117E1F31093B00D83
:1013220002C0E981ECB91881229608950E944516FF
:101332008BDFE03021F0A0915A08A03009F0C6C03E
:101342006CDF1E2FA091160DA53618F0E0E0E09399
:10135200120D3091120DE091120DE03059F411305E
:1013620019F4E4E0E093120D1A3519F4EBE0E0937E
:10137200120DA4C0E43089F4E0E0E093120D109362
:101382005B081093140DE6E0E093120DE0E0E093A9
:101392005A08E1E0E093130D91C0E53091F4E0E0EA
:1013A200E093120D0E948213E05DE11749F00E9462
:1013B20090140E9497140E949E14E6E0E093120D8E
:1013C2007DC0E63091F40E9497140E94901413306D
:1013D20049F4E7E0E093120DE0E0E093150D0E947E
:1013E200A41402C00E949E1469C0E73011F0E830D4
:1013F20059F41A93E5E1FDE0FA93EA93E2E1FDE0A4
:10140200FA93EA93CFDE5AC0E93081F4E0E0E09348
:10141200120D173131F4E091150DA091140DEA1758
:1014220009F003C0E4E5E0935A0848C0EB3069F4E0
:10143200103039F4ECE0E093120DE0E0E0935A084A
:1014420003C0E0E0E093120D39C0EC3049F4109390
:10145200170D1093140DE0E0E093130DEDE02CC096
:10146200ED3011F50E9497140E949E140E94901470
:10147200E091170DE150E093170DE030A1F4E091F7
:10148200140DE03069F4EEE0E093120DE091130DDB
:10149200E1500E94AC14A0E0A0830E94A41403C0F7
:1014A200E0E0E093120D0AC0EE3041F41D3019F471
:1014B200EAE5E0935A08E0E0E093120DE091120DA4
:1014C200E31719F0E0E0E093160D32CFDEC2AA93E3
:1014D200BA93EA93FA93EFB7EA931A930A931091A5
:1014E2009B0000919C00E12FEC71A9F4E0917A0E2F
:1014F200F0917B0EEE54F24F0083AAE7BEE00E9409
:101502009613E83CA0E0FA0731F4E0E0F0E0E09363
:101512007A0EF0937B0E09911991E991EFBFF9913F
:10152200E991B991A99118951A930E94B0140E9459
:10153200B514D9F30E94B014EE54F24F1081ACE707
:10154200BEE00E949613E83CA0E0FA0731F4E0E026
:10155200F0E0E0937C0EF0937D0EE12FB0C10E948B
:10156200B0140E94B51409F029C12AC10E9445167F
:10157200F6DFE03021F0A0910F0DA03009F08AC013
:10158200D3DF1E2FA091100DA53618F0E0E0E093F6
:101592000B0D30910B0DE0910B0DE03031F4113059
:1015A20019F4E4E0E0930B0D6DC0E430C1F4E0E027
:1015B200E0930B0D1A3229F00E948213E05DE117CD
:1015C20069F410935B0A10930D0DE5E0E0930B0DA7
:1015D200E0E0E0930F0DE1E0E0930C0D53C0E53045
:1015E200A9F4E0E0E0930B0D0E948213E05DE117A5
:1015F20061F00E94BC140E94C314E0910C0DEF5FD5
:10160200E0930C0DE6E0E0930B0D3CC0E630D1F424
:101612000E94C3140E94BC14133071F4E7E0E093FB
:101622000B0DE0E0E0930E0DE0910C0DF0E0E55AB9
:10163200F54FA0E0A08305C0E0910C0DEF5FE093B1
:101642000C0D20C0E73011F0E83059F41A93EEE0A7
:10165200FDE0FA93EA93EBE0FDE0FA93EA93A2DD70
:1016620011C0E93079F4E0E0E0930B0D173131F469
:10167200E0910E0DA0910D0DEA1709F003C0E4E50B
:10168200E0930F0DE0910B0DE31719F0E0E0E0930A
:10169200100D6ECFFAC1AA93EA93FA93EFB7EA93C9
:1016A200E091810FA091800FEA1781F0E091590833
:1016B200E03019F0E89421F808C00E94CA140E9490
:1016C200D81419F4E0E0E093810F03C0E89420F805
:1016D20021F8E991EFBFF991E991A9911895E88173
:1016E200A091110DEA0FE093110DE091800FF0E04F
:1016F200E058F14FA881A083E091800FEF5FE09363
:10170200800F0E94D81419F4E0E0E093800FB6C075
:10171200E0E0E093810FA091800FA13020F00E94C1
:10172200CA14689421F80895AA93BA93EA93EFB77A
:10173200EA93E0E0E093810F0E948213EF5FE0936F
:101742005908E991EFBFE991B991A99118950E94C1
:10175200B713A03220F00E94B713AB3309F403C0D1
:101762000E94C413F4CF0E94B713AB3311F40E944A
:10177200C41308950E94B713E881EA1729F40E945E
:10178200C4133197E1E07AC0E0E078C00E94B71359
:10179200A03228F00E947214E181E03208F410C0F5
:1017A2000E947A14EC91E0935C0B0E94C4130E9495
:1017B2007A14EC91E0935D0B0E94C413E1E008956A
:1017C200E0E008951A930A9310E00E947A140C91B3
:1017D2000B3311F0003208F412C0013310F0093358
:1017E20008F007C0E02FE053F0E0E457FF4FE49128
:1017F2001E2B0E94C4130E947A140C91E9CFE12F90
:101802000991199108950E94451600E010E00E9486
:10181200B713AD3229F40E94C4132FEF3FEF02C079
:1018220021E030E00E94B713A03320F00E94B713EA
:10183200AA3308F00FC0D801EAE0F0E00E94B81520
:101842000E940C14E053F0E0E00DF11D8F010E94A4
:10185200C413E8CFF901D8010E94B81516C1E88176
:101862000E945214E881A091770BEA0FE093770B64
:10187200E881A091780BEA27E093780B21960895EE
:101882001A9310E00E94DD14E03031F00E94DD1462
:10189200EA93E5DF1F5FF6CF2BC01A9310E00E9498
:1018A200F013E25AF44FE081E03049F00E94F01365
:1018B200E25AF44FE081EA93D2DF1F5FF0CF199131
:1018C20008950E941814E6EBF2E0FA93EA93EC8191
:1018D200FD810E94E5140C94DF101A930E941814E3
:1018E200E9EBF2E0FA93EA93ED81FE810E94E514BE
:1018F2001881239608951A93ECE3EA93B0DF11E07E
:10190200193080F40E94F013E457FF4FE491A9814B
:10191200EA2319F0E12FE05D01C0E0E2EA939FDFE4
:101922001F5FEECFEEE3EA939ADF0C94DE101A9378
:101932000A93E0915B09E03011F40C941D11EAE581
:10194200EA93CBDCE0E0EA93C8DC10E00E94F013FB
:10195200E55AF64FE081E03011F01F5FF7CF1F5FCD
:10196200012F0A93BADC10E00E94F013E55AF64FF9
:10197200E081E03079F00E94F013E55AF64FE08101
:10198200EA93ABDC0E94F013E55AF64FE0810E0FAA
:101992001F5FEACFE02FE195EA939FDCEDE0EA9347
:1019A2009CDC0C941D110E944516AC81BD81EC910A
:1019B200E03021F40E944C160C948411E0E0E09394
:1019C200800FE1E0EA938BDEE0E0E093110DAC8161
:1019D200BD81EC91E03041F0EA9381DEEC81FD8142
:1019E2003196EC83FD83F3CFE3E0EA9378DEE09176
:1019F200110DE295EF70EA930E9429040E2FE091F7
:101A0200110DEF70EA930E9429043E2F0A9367DEBC
:101A12003A9365DEE7E1EA9362DE689420F80E9479
:101A22004C160C9484110E94451680DCA0915A0831
:101A3200AA3511F40E945208A0915A08A43511F552
:101A420000E00E943414EB5FFA4F9F01E02F0E94E6
:101A5200AC14E081E03051F0E02F0E94AC14E08140
:101A6200D901EC930F5F2F5F3F4FF0CFD901E0E038
:101A7200EC930E9434140E94EF14E0E0E0935A08C1
:101A8200E12F03C0E0E0E0935A080E944C1624962E
:101A920008950E9443166ADDA0910F0DA43511F03E
:101AA2000C94D60D10E0A0915B0AAA3221F4E091C9
:101AB2005D0AED3409F059C0E7E0E093E10CE091F2
:101AC2005E0AEA3511F00C94A80D00E04FEF5FEFCB
:101AD200E091600AE7703E2FE0915F0AE23361F421
:101AE200A4E1B0E00E941A16AE2F0E94CD13E45773
:101AF200FF4FE491EA2309F414C0E1E6FAE00E9400
:101B02006D140E94B713AB3421F40E94C4137BDE20
:101B12000E2F0E94B713A43521F40E94C41373DE62
:101B2200AF0100930005E8ECF0E0E093950BF09331
:101B3200960B4093E50C5093E60CE2E0E093E10C47
:101B4200E0915F0AE93319F4E1E0E093E10CE091FE
:101B52005E0AE03519F4E1E0E093E10CE0915E0AFF
:101B6200E23419F4E1E0E093E10C0E948213E05DBB
:101B7200A0915B0AEA1799F4E0915D0AE23521F43B
:101B82000E9419081E2F0BC0E23721F40E94BF07E2
:101B92001E2F05C0EA3519F40E949B081E2FE0E0B3
:101BA200E0930F0DE12F0C948211E0E00C9482116E
:101BB200A0E020FCA1E0A13049F4A0E021FCA1E0DA
:101BC200A03021F4A0915908A03009F001C0A0DD95
:101BD200E0915908E03019F0E150E0935908089576
:101BE200A881A13118F0E881E051E883E8810E94E0
:101BF200FB14A091DC0FB091DD0FEA2BFB2BE093DD
:101C0200DC0FF093DD0F0C94B1111A930A9310E0DC
:101C12001031D0F40E94F0130E94E513AFEBBBE049
:101C2200EE27A10FBE1FEC93AFECBBE0EE27A10F96
:101C3200BE1FEC93AFE0BCE00E94F0130E940515BA
:101C42000E940A151F5FE4CFF7C20E944516E09179
:101C52007D0BF0917E0BAC81BD81EA27FB279F01B2
:101C620010E0123190F4F901E17039F0A12FB0E0E7
:101C7200A058B44FEC91EF5FEC93D901E2E0F0E0B1
:101C82000E94DE159F011F5FECCFEC81FD81E09386
:101C92007D0BF0937E0B0E944C1635C30E946504A7
:101CA200E03061F10E943414EB5FFA4F0E94681435
:101CB200AFEABBE0E881F0E0AE0FBF1FEC910E94FB
:101CC20052140E948213E05D0E9452140E94281452
:101CD200E2E50E944E140E940F150E945414E4EC97
:101CE200F2E00E94B313E8810E941B150E94D013F8
:101CF2000E9457140E9434140E94EF140C94B111E4
:101D02000E946504E03069F10E943414EB5FFA4FDF
:101D12000E946814A5E1B0E00E941A16E05D0E94DC
:101D220052140E948213E05D0E9452140E942814F1
:101D3200E2E50E944E140E940F150E945414E7EC33
:101D4200F2E00E94B313E9810E9421140E94D6138B
:101D5200E8810E9421140E9457140E9434140E94A8
:101D6200EF142CC20E944316A091950BB091960BD2
:101D72000E943F1624F4A5E9BBE00E942015E091E1
:101D8200950BF091960B309719F4E0E0E093000583
:101D920010E0123110F00C94180FA12FB0E0AF5FD9
:101DA200BF4F0E941A16E13011F00C94160F0E94D8
:101DB200F013E653F04F0081E12FE695E695E695A4
:101DC2002E2FE12FE770EF5F5E2FE22FF0E0EE564D
:101DD200F44F1080E52F0E94FB14A12DB0E0EA23FE
:101DE200FB233097B9F40A3821F40E946504E030ED
:101DF20009F406C0E12FEF5FEA93E0E0EA9380DFA7
:101E0200003810F00B3808F001C00F5F003209F4FF
:101E120000E806C0003208F40F5F013808F000E065
:101E22000E94F013E653F04F00831F5FB2CFE0E051
:101E3200F0E0E093DC0FF093DD0FE093E40C00E0C0
:101E4200003110F00C94E30FE02F0E941B15E030DC
:101E520031F0AFECBBE00E942615E07809F0B0C08B
:101E6200E091E40CEF5FE093E40CAFEDBBE00E9485
:101E72002615E03079F40E942B150E9405150E9468
:101E820020150E942B150E94DA13309711F40E943C
:101E920030158CC0E13011F00C94B30F0E9436154E
:101EA200E1501E2F0E94F013E058F44FE081E03021
:101EB200A9F40E9439150E9496130E943E1530978C
:101EC20049F00E9439150D901C900E943E15E015B4
:101ED200F1050CF002C00E9430151BC00E942B15A8
:101EE2000E944315BF010E942B150E94DA13DF01E5
:101EF2000E94F0130E9448150E949C13DB01ED938F
:101F0200FC930E94F0130E944D150E9439150E9405
:101F12000A150E942B150E94DA13FF2332F40E9445
:101F22002B150E9405150E940A150E942B150E946E
:101F3200DA13309711F40E9430150E9452150E9454
:101F4200DA13309771F00E9452150E9405150E9413
:101F520020150E9452150E94DA13309711F40E9444
:101F6200301524C0E23011F50E943615E1501E2FC3
:101F72000E9457150E9443150F010E9457150E9497
:101F8200DA13DF010E94F0130E944815EA0FFB1FCB
:101F9200D001ED93FC930E94F0130E944D15AFE423
:101FA200BCE0E02F0E945C150E9496130E94361539
:101FB200EA9316DEAFEFBBE00E942615EA9310DE2D
:101FC2000F5F3ECFE091DC0FF091DD0FE093DF0C6D
:101FD200F093E00C96C10E94451630E010E01031FB
:101FE20068F40E94F013E156F44FE081AE2FEC81C9
:101FF200EA1711F431E002C01F5FF1CF303071F403
:1020020010E0103158F40E94F013E156F44FE081D1
:10201200E03011F431E002C01F5FF3CF313011F034
:102022000C94B010A091E20CA130A1F0E0919B0BB6
:10203200F0919C0B309721F4E0E00E944C1663C1B2
:10204200AFEDBBE00E94F013EA0FFB1FA091990BCA
:10205200A08307C0AFEDBBE0EE27A10FBE1FE2E0F9
:10206200EC93A091970BA13118F0E0E0E093970B6D
:10207200A091980BA13118F0E0E0E093980BAFEE3D
:10208200BBE00E94F013EA0FFB1FA091970BA08305
:10209200AFEFBBE00E94F013EA0FFB1FA091980B79
:1020A200A083AFEEBBE0EE27A10FBE1F2C91213023
:1020B20068F0E22FE150F0E00E944D15E22FE1506E
:1020C200A6EABFE00E945C150E940A15AFE0BCE0E0
:1020D2000E94F0130E944315A0919B0BB0919C0BA0
:1020E200A083B183AFE2BCE00E94F0130E944315CB
:1020F200A0919D0BB0919E0BA083B1830E94F0131F
:10210200E156F44FAC81A083AFEBBBE00E94F01329
:10211200EA0FFB1FA091E70CA083AFECBBE00E948B
:10212200F013EA0FFB1FAD81A083AFE4BCE00E9475
:10213200F0130E9405150E940A15AFE6BCE00E944A
:10214200F0130E9405150E940A15AFEABBE00E9437
:10215200F013EA0FFB1FA0919A0BA08331E0E32F4B
:102162000E944C16D0C01A9310E0103488F4E12F6C
:10217200AFE9BBE00E945C150E940A15AFE1BCE02A
:102182000E94F0130E9405150E940A151F5FEDCFF1
:1021920010E0123130F40E94F0130E944D151F5FBF
:1021A200F8CFE981E03009F406C0A091E30CAF5FFB
:1021B200E3E00E94E315E093E30C18812296089570
:1021C20024DD0C94B1111A930A93E091E20CA091D0
:1021D200E10CEA1789F00091E10C073009F415DDF2
:1021E200013019F4E0E0EA93BEDF023019F4E1E0D5
:1021F200EA93E6DF0093E20CA091E20CA73019F417
:10220200E0E0E0937F0BA091E20CA13019F4E0E052
:10221200E0937F0BA091E20CA23071F4A091000533
:10222200A13020F0A091E60CAA230AF402C0E1E05A
:1022320001C0E0E0E0937F0B0991199108950E949B
:102242004316E7E0E093E10C10E0153110F00C9436
:1022520082110E94F0130E94131432960E940616F5
:102262009F010E94F0130E94131432960E940616D8
:10227200AF010E94F0130E9413143496E491E030EF
:1022820011F0E130B1F4D9010E941A16AE2F0E946A
:10229200F0130E9413143596E491EA1748F40E9451
:1022A200F0130E9413143696E491D9010E942E165F
:1022B20026C0E230A1F4DA010E941616E031A7E24C
:1022C200FA0714F4FF2352F40E94F0130E9413142D
:1022D20036960E940616DA010E94261610C0E330D6
:1022E20071F4D9010E941A16EF3F49F40E94F013CB
:1022F2000E9413143696E491D9010E942E161F5F94
:10230200A4CF0E944A1626960895E991F991A991BF
:10231200B9911D900590011421F40020D1F7EE2708
:1023220008951018E1F3E1E008F4E2500895A9914C
:10233200B991EE27FF276D91662311F03196FBCFFD
:102342000895AA27BB27E991F9910590002011F081
:102352001196FBCFFD0108955D9BFECFE881ECB99C
:10236200219608951A930A93AC81BD810E940216A8
:102372003097C1F0AA81BB810E9402168F0130976B
:1023820049F00230E0E01E0760F0F80131978F015A
:10239200ED93FC93AC81BD810E9496133197AE817F
:1023A200A08303C0EE81EA93D7DF198108812796C3
:1023B200089526970E94431610E0EA89FB89319618
:1023C200EA8BFB8B3197E4912E2FE03011F40C94C1
:1023D2000613E12FE03039F4253211F411E002C086
:1023E2000E945E1511C1E130A9F4253219F40E9450
:1023F2005E1509C112E040E000E02D3211F401E067
:1024020003C12B3211F44BE2FFC0203211F440E23F
:10241200FBC002C0E23039F450E013E0203311F483
:102422000068F2C004C0E33011F00C9405132033AD
:1024320010F02A3308F009C0A52FEAE0EA9FF00164
:102442005E2FE22FE0535E0FDFC0E22FE33649F446
:102452000E946915E889F989A481AA930E946F15DF
:10246200D2C0E33741F40E9469150E9479150E9497
:1024720098111E2F0AC0E03761F40E9469150E946C
:1024820079150E94A2111E2F086002600F7730E0BA
:1024920035C0E43611F0E93611F4046002C0E537C4
:1024A20031F4E6E3F2E0EE83FF8315E00DC0E83598
:1024B20011F4086004C0E83711F00C940413E0E44E
:1024C200F2E0EE83FF8314E002FF14C00E9469155C
:1024D2000E948315AB85AA233AF4EA85FB850E9404
:1024E2009B15EA87FB874DE2403011F01F5F01C068
:1024F2000B7F04C00E9469150E94831500FD11C064
:10250200151778F407FF08C002FF04C00B7F242FC1
:10251200115001C020E301C020E20E945E1551501B
:10252200EFCF312F01FF1AC03030B9F003FF08C0DE
:10253200EE81FF813196EE83FF833197E49105C0EE
:10254200AE81BF81ED91AE83BF83EA930E946F1586
:10255200503009F051503150E7CF4BC020E3EE81AB
:10256200FF810E940616E887F987EE81FF81329685
:10257200EE83FF83E885F985AA85BB85AE17BF0781
:1025820050F02F5FA885B985EA85FB85EA1BFB0B16
:10259200EA87FB87EFCF2A3328F003FF02C0295FC7
:1025A20001C0295D04FD1AC0213320F4A885B98534
:1025B200119709F409C0531710F000FF01C013C0AE
:1025C20020E207FF0BC020E3006102FF07C00B7F80
:1025D2004A930E946F15503009F051500E945E15C7
:1025E200503009F051503150A885B985129708F042
:1025F200B5CF00FF08C0503031F05150E0E2EA930D
:102602000E946F15F8CF10E0D8CE0E944A16649649
:102612000895FF92F82E22971A930A93DE010E94E0
:1026220097158D01DE0116960E9497150E940216DB
:10263200EA83FB83DE0114960E9497150E9402161C
:10264200FA93EA931A930A93FE013696FA93EA935F
:10265200E0E0F0E0FA93EA93ACDEAA81BB81E0E02D
:10266200EC93198108812496FF9008950A921A9298
:10267200FA926A937A938A939A93AA93BA93EA9371
:10268200FA93EFB7EA930895E0915206EA930E9413
:102692005B04E09352060895EAE0F0E0FA93EA93CD
:1026A2000895E0915206A3E4EA9FF0010895EB5FDA
:1026B200FA4FFA93EA930E94D40CF3CFEE5FFA4FEB
:1026C200A0E0A083E1CFEA930E942904EA930C944C
:1026D2008F04E8EEFCE0E093060DF093070D0895F9
:1026E200A091060DB091070D0895A091060DB0912D
:1026F200070D1796EC930895AF5FE4E60E94E31589
:102702000895A0E0B0E00E941A160895E8ECF0E007
:10271200FA93EA930C948B15EA930E94A301E6E9DB
:10272200F0E0FA93EA930C948B15ED91FD913196BA
:10273200FE93EE9308950E940F16EA1BFB0B089579
:10274200E881F981FA93EA930E94620CECE2EA933F
:102752000C94300CFA93EA930E94620CEBE3EA9336
:102762000C94300CFA93EA930C94410CA0917B0BDD
:10277200B0917C0BAC910895A0917B0BB0917C0B36
:10278200EC91EA930895ABE7BBE0CFCF0E94040C33
:10279200E058FF4F1E2F0895E32FF0E00895EF77E2
:1027A200F0E0FA93EA930C94620CEAE3EA930C9455
:1027B200300CEE0FFF1FAE0FBF1F0E9402160895CE
:1027C200FA93EA930C94620CE156F44FA0E0A083D2
:1027D2000895EAE3EA930E94BB0BE1300895E12FEA
:1027E200F0E00895EA0FFB1F0F01AFECBBE0EE270C
:1027F200A30FBE1FEC910895F0E0FA93EA930E94B2
:102802006E0CD3CFA091790BB0917A0BE0E0EC93F0
:102812000E944A1608950F01A0917B0BB0917C0B88
:10282200EC9108950E949F15EA56FF4F0895EEE538
:10283200FBE0FA93EA930895E0915B0BF0E0F2CFAC
:10284200F0E0BECF32960E940616DF010895A091F5
:10285200790BB0917A0B0895E0E6FAE0E0937B0BF6
:10286200F0937C0B0895E0915106A3E4EA9FF001F6
:102872000895EB5FFA4FE093790BF0937A0BE091B6
:102882005C0AE5DFEC93A9E7BBE04FCFE0915B0A7E
:10289200DEDFEC93A9E7BBE048CFEC93A9E7BBE00E
:1028A20044CFD5DFFACFD3DFEFE0F7CFD0DFE0E0E0
:1028B200EC930895EE5FFA4FA1E0A083E0915106F8
:1028C200EA930E945B04E0935106E1E00895E093ED
:1028D200790BF0937A0B0895E0937B0BF0937C0BCA
:1028E2000895E0917B0BF0917C0B0895A9E7BBE082
:1028F2001CCFA0917B0BB0917C0B0895AA81BB8168
:10290200EC91E295E07FAE2FEC810895EA0FAA8167
:10291200BB81EC93A881B981EC91EF5F0895E12F1F
:10292200A091140DEA0FE093140D0895E091130D98
:10293200F0E0E55AF74F10830895E091130DEF5F31
:10294200E093130D0895E091130DF0E0E55AF74F6F
:10295200A0E0A0830895F0E0E55AF74F0895E091D2
:102962007C0EF0917D0E0895A0917A0EB0917B0EAF
:10297200EA17FB070895E12FA0910D0DEA0FE093EE
:102982000D0D0895E0910C0DF0E0E55AF54F10831E
:102992000895E091810FF0E0E058F14FE081E0937B
:1029A2009C00E091810FEF5FE093810F0895F0E0CA
:1029B200E030A1E0FA070895E12FA981BA81F0E0A1
:1029C200EA0FFB1FE49108950E94AB150E940A16BC
:1029D20084E00E940A1328960C944E0CEE5FFA4F84
:1029E200A1E0A083E0915106EA930E945B04E09388
:1029F20051060895A6E4B1E0F0E0EE0FFF1FEA0FE2
:102A0200FB1F0E9406160895EE0FFF1FAE0FBF1F99
:102A12000895E0E0F0E0ED93FC930895E09156060E
:102A2200E05D15DFEC93E0915606EF5FE770E0930F
:102A320056065CCFF0E0E156F44FE0810895ED9147
:102A4200FD913197FE93EE930895EE27A00FBE1FDE
:102A5200EC910895AFE0BCE0E02FF0E008950A9316
:102A62000E944F0EE02FF0E0AFCEAFEEBBE0EDCF15
:102A7200E12FA6EABFE0F0E0C7CFE12FA2E8BFE076
:102A8200F0E097CEEE0FFF1FEA0FFB1F0895E0580C
:102A9200F44FE081F0E00895E058F44FA0E0A08305
:102AA2000895AFE2BCE0E02FF0E00895AFE6BCE0AD
:102AB200E02FF0E00895F0E0A7CF2A93EF85F889A0
:102AC200FA93EA93FE013F96FA93EA930C94B311B8
:102AD200E889F9893497E88BF98B0895EF85F889AD
:102AE200FA93EA93FE013F96FA93EA930C94B31198
:102AF200A889B98914960E940216EE83FF83FA937D
:102B0200EA930895A889B98914960E940216EA8761
:102B1200FB870895E991F991309639F080EA9FE0B8
:102B22000197F1F7A8953197C9F708950024AF0DE1
:102B3200B01D0895F195E195F0400895EE0FFF1F45
:102B4200EE0FFF1FEE0FFF1F0895EF2FFF27E7FD88
:102B5200FFEF08956F2F660F660B762F0895FA9F89
:102B6200F02DEB9FF00DEA9FE02DF10D08953BD083
:102B7200F6DF0EF4DFDF0895002498E0AA0F001CB0
:102B82000E1A10F40E0E01C0A1609A95B9F7EA2F41
:102B9200A02D08950024112490E1AA0FBB1F001C50
:102BA200111C0E1A1F0A18F40E0E1F1E01C0A1607E
:102BB2009A9599F7FD01D001089515D0EBDF0EF437
:102BC200B9DF0895D9DFEA2F0895E894B7FF04C06A
:102BD200A095B09511966894F7FDACDFDBDFFD019F
:102BE2000EF4A8DF0895E894F7FF02C0A3DF68940B
:102BF200B7FF06C0A095B095119600F8039400FAAD
:102C02000895ED91FC91119708950590F491E02DAE
:102C120008957A936A93FA93EA9308951B2EBF2F2D
:102C2200F12D1A2EAE2FE12D0895119602D0FE2F0E
:102C32001197E199FECFFF93FFB7F894AEBBBFBBEC
:102C4200E09AEDB3FFBFFF91089507D01196EF937D
:102C5200EF2F03D0EF9111970895E19B02C0A89541
:102C6200FCCF9FB7F894AEBBBFBBE09A8DB3E81719
:102C720019F0EDBBE29AE19A9FBF089500240A166B
:102C82000B0608955A934A933A932A931A930A93F6
:102C920008955D814C813B812A81198108810895C3
:00000001FF
